:0300000002352B9B
:0C352B0078FFE4F6D8FD75815D02357272
:10104A000A53746172743A20004950436F6E6E6598
:10105A0063745245510A00444843502D4F4B0A00CD
:10106A004950436F6E6E656374003E432C562C43A1
:10107A00432CC0E4E0EFF2E5F020D1E8EDEAEEEC33
:10108A0049500A003E432C4D41432C2530326258C8
:10109A003A25303262583A25303262583A2530328F
:1010AA0062583A25303262583A25303262582C4D0D
:1010BA00414320E0E4F0E5F10A003E432C56455254
:1010CA002C20332E3020EEF22025732025732CC2DB
:1010DA00E5F0F1E8FF20495020ECEEE4F3EBFF0ADB
:1010EA000041707220303420323030370031303ACB
:1010FA0030343A3532003E432C4C442C50524F4740
:10110A003A202020202020202020202020202020BB
:10111A0020202020202020202020202020202020C5
:10112A0020202020202020202020202020202020B5
:10113A0020202020202020202020202020202020A5
:10114A002020202020202CC4E0F2E020E7E0EFE875
:10115A00F1E82028F4E0E9EB290A003E2A2C312C98
:10116A00C1E0E7EEE2FBE520EFE0F0E0ECE5F2F0CB
:10117A00FB20F1E5F2E5E2EEE3EE20E8EDF2E5F040
:10118A00F4E5E9F1E00A003E412C4130312C2562B8
:10119A00752E2562752E2562752E2562752C49508D
:1011AA0020E0E4F0E5F120E0E4E0EFF2E5F0E00A27
:1011BA00003E412C4130322C2562752E2562752E57
:1011CA002562752E2562752C495020E0E4F0E5F180
:1011DA0020EEF1ED2E20F1E5F0E2E5F0E00A003E26
:1011EA00412C4130332C2562752E2562752E2562DD
:1011FA00752E2562752C495020E0E4F0E5F120F0C7
:10120A00E5E72E20F1E5F0E2E5F0E00A003E412CA8
:10121A004130342C2562752E2562752E2562752E75
:10122A002562752CCCE0F1EAE020F1E5F2E80A004B
:10123A003E412C4130352C2562752E2562752E25AE
:10124A0062752E2562752CD8EBFEE70A003E532CF8
:10125A004130362C2562752CCCE0EAF12E20E7E0ED
:10126A00E4E5F0E6EAE020EFE0EAE5F2E020E22059
:10127A00F1E5F2E820282A3130ECF1290A003E2A69
:10128A002C312CC4EEEF2E20EFE0F0E0ECE5F2F08A
:10129A00FB20F1E5F2E5E2EEE3EE20E8EDF2E5F01F
:1012AA00F4E5E9F1E00A003E422C5330312C256284
:1012BA00752CCFE0F1F1E8E2EDEEE520F1EEE5E4A0
:1012CA00E8EDE5EDE8E520F120F1E5F0E2E5F0EE04
:1012DA00EC0A003E422C5330322C2562752C43E234
:1012EA00FFE7FC20F120F1E5F0E2E5F0EEEC20ED7D
:1012FA00E520EFEEE4E4E5F0E6E8E2E0F2FC0A00DD
:10130A003E422C5330332C2562752CCFE5F0E5E7AD
:10131A00E0EFF3F1EA20EFF0E820EFEEF2E5F0E596
:10132A0020F1E2FFE7E820F120F1E5F0E2E5F0EE56
:10133A00EC0A003E422C5330342C2562752CC7E04F
:10134A00EFF0E5F2E8F2FC20EFE5F0E5E4E0F7F390
:10135A0020E4E8E0E3EDEEF1F2E8EAE820E220F149
:10136A00E5F0E2E5F00A003E422C5330352C2562C6
:10137A00752CCAE0EDE0EB20F8E8F0EEEAEEE2E5E3
:10138A00F8E0F2E5EBFCEDEEE3EE20EEE1ECE5ED64
:10139A00E00A003E532C5330362C25303262582551
:1013AA003032625825303262582530326258253040
:1013BA0032625825303262582C4D414320E0E4F025
:1013CA00E5F120F8E8F0EEEAEEE2E5F8E0F2E5EB26
:1013DA00FCEDEEE3EE20EEE1ECE5EDE00A003E4541
:1013EA004E440A0044756D70582020202020303069
:1013FA002030312030322030332030342030352034
:10140A0030362030372030382030392030412030F3
:10141A00422030432030442030452030460A003AEA
:10142A0020000A0044756D704420202020203030AE
:10143A0020303120303220303320303420303520F3
:10144A0030362030372030382030392030412030B3
:10145A00422030432030442030452030460A00459F
:10146A007272206B657900526420656570726F6DC7
:10147A000A005264204D454D0A00526420436F64AD
:10148A00650A0044656275674950204F4E0A004458
:10149A00656275674950204F46460A004465627581
:1014AA006755736572204F6E0A0044656275675509
:1014BA00736572204F46460A0044656275674D732C
:1014CA0067204F6E0A0044656275674D7367204F47
:1014DA0046460A00436F6E666967206C6F636B212C
:1014EA000A00577220656570726F6D0A0020536199
:1014FA00766520656570726F6D210A0045727220EB
:10150A004D414321004C6F61643E3E002A003C413C
:10151A0030313D003C4130323D003C4130333D00EA
:10152A003C4130343D003C4130353D003C41303691
:10153A003D004E4F4950004C494E4B434F4E54527A
:10154A00005452415353004652004E4F4C494E4BA1
:10155A0000494E49004E4F4449414700003C210092
:10156A003C5330313D003C5330323D003C53303324
:10157A003D003C5330343D003C5330353D003C5334
:10158A0030363D00FF153CFF1541FF154BFF155145
:0C159A00FF1554FF155BFF155FFF156681
:063ED400010B00010900D2
:103E9000C2AFC28E758900438910758BFF758DB7CF
:073EA000D2ABD28ED2AF229B
:03001B00023400AC
:10340000C0E0C083C082C0D0C2AFC28E758BFF75D2
:103410008DB720060675A61E75A6E10509D202E540
:103420000B6002050BE50AD394014002150A050E54
:10343000E50E540F704AD20DE50E543F7014D200C1
:1034400090668DE0600C04F0E0D394B44004C2AF09
:1034500080FE906688E0600204F0906104E0600203
:1034600014F090668EE0D394014003E014F0300530
:1034700002050CE50DD394644004D2068002050DCC
:10348000E508D3940140021508D28ED2AFD0D0D037
:0634900082D083D0E0327F
:10083E00C291C290C2B5C20A7D027C007F07123EF1
:10084E00248F25E525646060097D017F60123DB827
:10085E00D20AE4FDFC7F0B123E248F25E52530E6FF
:10086E00097D04E4FF123DDCD20A7D017C007F0786
:10087E00123E248F25E5257008FD7FFF123DB8D26C
:10088E000A300A03126000C2AFC288C2A8C2AA12FE
:10089E0037C0906341E0B4FA09A3E064CE7003025E
:1008AE000935E4F52574392525F582E43463F5839D
:1008BE00E4F00525E525B443EC90634174FAF0A30A
:1008CE0074CEF0A374CCF0906347740AF0E4A3F0F6
:1008DE00A304F0A3F090634C7403F0A374CCF090D7
:1008EE00633D74FFF0A3F0A3F0E4A3F0906358749B
:1008FE0005F0E4F525E5252401FFE433FE743925E2
:10090E0025F582E43463F583E0FD123E770525E597
:10091E0025C3944340DFE4F5A775A61E75A6E190A6
:10092E007FF0F0A3F080FED2AF90634C7403F0A37F
:10093E0074CCF0E490634BF0122C74EF6003121D34
:10094E009DD2B51230BAC206123BFB906358E0C37B
:10095E00940350037403F0D20CD20BD20AD293201C
:10096E000A077E107F4A122D5AE4906578F0123EE7
:10097E0090C2AFA37408F09062B77424F0E4A3F0B1
:10098E00906341E09062B9F0906342E09062BAF0F9
:10099E00906343E09062BBF0906344E09062BCF0E1
:1009AE00906345E09062BDF0906346E09062BEF0C9
:1009BE00750A01E490657AF0C207C208D2AF75A736
:1009CE000775A61E75A6E1123D92200A19AF257E67
:1009DE00007D03122E3BE4FF1231727E637F78E4BA
:1009EE00FB7D01122F1590668DE060037401F0E41B
:1009FE00906104F0A37455F0A37481F0E4F50CE457
:100A0E00F50D906104E07003121B7390668EE0B4D6
:100A1E0001119080007410F0E490668EF0D20AD22C
:100A2E000BD20C908008E0F52530E405D207741047
:100A3E00F0E52530E508D2099080087420F0E52510
:100A4E0030E608D2089080087440F0E50CD3940389
:100A5E00402D908002E4F0908001F0908000F0E54F
:100A6E000CD3940440037401F0E50CD39406400FAC
:100A7E00E4F50CC20390657AF0750A01123BFB9007
:100A8E0080A0E070031238B99080B8E07003123283
:100A9E00BF9080D0E07014300E1190668474FFF019
:100AAE0090634CE0FEA3E0FF123AE9908000E07004
:100ABE0013300710122B70906334EFF0D394004074
:100ACE0003120026908002E07006908000E0600520
:100ADE00D205020A0DC205E4F50C906104E0600334
:100AEE00020A0D3009121227B5906334EFF0D39439
:100AFE00004005E0FF123EA7200803020D12122649
:100B0E0040906334EFF07003020A0D90668DE06042
:100B1E00037401F0906378E054BF247F7003020BDE
:100B2E00E6147003020BC724026003020CBD200AF8
:100B3E00077E107F53122D5A906350E0700690631B
:100B4E0054E0605B906684E0FF906350E0B507244C
:100B5E00906685E0FE906351E0B50618906686E0DB
:100B6E00FE906352E0B5060C906687E0FE906353EC
:100B7E00E06E602B906354E06F7035906685E0FFF9
:100B8E00906355E0B50729906686E0FF906356E0C6
:100B9E00B5071D906687E0FF906357E0B50711C259
:100BAE000390657A7403F0120021750A01020D128A
:100BBE0090668474FFF0020D1290667CE0FF9063E5
:100BCE007AE06F6003020D1290667CE004F0E4F5AB
:100BDE000A906578F0020D12300303020D12906335
:100BEE0079E0D3940A5003020C90A3E064026003F0
:100BFE00020C90906341E0FF906383E06F6003020C
:100C0E000A0D906342E0FF906384E06F6003020A76
:100C1E000D906343E0FF906385E06F6003020A0D61
:100C2E00906344E0FF906386E06F6003020A0D90CC
:100C3E006345E0FF906387E06F6003020A0D9063E7
:100C4E0046E0FF906388E06F6003020A0D7E107F1E
:100C5E0061122D5A90637B63A20190633963A201E6
:100C6E007F1212222290638D63A20190668463A28A
:100C7E00017F0412222290657A7406F0750A020230
:100C8E000A0D744744637003020A0D123EDBD20351
:100C9E00E4F50A906578F090668804F0E490667B3F
:100CAE00F0A3F0200A5E7E107F6A122D5A80553016
:100CBE000352906378E020E74B90637AE0FF9066F2
:100CCE007BE0FE6F600D906683E07007EE146F7030
:100CDE0033801390667BE004F0906334E0FFD3948E
:100CEE00044003122A4F9060007482F0A37401F046
:100CFE0090637AE0906002F07E607F007D03123890
:100D0E003E020A0D200303020DDB9080D0E0700E30
:100D1E0090634CE0FEA3E0FF123AE9020A0DE50AE9
:100D2E00706B1239ACEF60207E647F78906479E04E
:100D3E002404FD12383E906683E06003020A0D9093
:100D4E006358E0F50A020A0D906688E0D3943C40A1
:100D5E003C906683E0703690668804F09062B6E050
:100D6E00702B123EC1E4906478F0A37412F090667A
:100D7E007CE090647AF0A374FDF090610763A201A9
:100D8E0090647C63A2017F12122222809B123EB6D7
:100D9E00EF60159060007483F0E4A3F07E607F0036
:100DAE007D0212383E020A0DE50A64016003020A52
:100DBE000D906578E004F0E0C394055003020D3603
:100DCE00C203E490657AF0120021020A0DE50A646E
:100DDE00016003020A0D90657AE0147003020E7131
:100DEE00147003020E9D147003020F45147003025B
:100DFE000FFB24FE605B24066003020A0DE4F50C73
:100E0E00F52574B02525F582E43461F583E0FF7491
:100E1E00392525F582E43463F583EFF00525E525C4
:100E2E00B43FDF200E1390657A7404F0906578E07D
:100E3E005401F0750A01020A0D90657A7404F0905F
:100E4E0065787401F0750AC890668474FFF0020A22
:100E5E000DE4F50C123BFB90657A7401F0750A03F4
:100E6E00020A0D906684E0600B90634CE0FEA3E0F6
:100E7E00FF123AE9750A0290657A7402F0906347A0
:100E8E00E07003020A0D90657A7403F0020A0D9069
:100E9E006684E07003020F369064787480F090647C
:100EAE007A7402F0E4A3F0A304F090634163A2010C
:100EBE0090647D63A2017F0A1222229064877430AF
:100ECE00F0A3747BF0E4F525742F2525F582E43428
:100EDE0061F583E0FF601174892525F582E43464A1
:100EEE00F583EFF0052580E074892525F582E4343D
:100EFE0064F583747DF0748A2525F582E43464F5F7
:100F0E0083E4F0E5252411906479F07C667D84906D
:100F1E00634CE0FAA3E0FB7F0212363C7E647F78DE
:100F2E00E5252413FD12383E90657A7404F0906323
:100F3E0058E0F50A020A0D906684E07003020FEC89
:100F4E009064787480F090647A7401F0E4A3F0A356
:100F5E0004F0A37430F0A3747BF0E4F525742F2510
:100F6E0025F582E43461F583E0FF6011747F252559
:100F7E00F582E43464F583EFF0052580E0747F2577
:100F8E0025F582E43464F583747DF074802525F5AF
:100F9E0082E43464F583E4F0E5252407906479F067
:100FAE007C667D8490634CE0FAA3E0FB7F021236F0
:100FBE003C7E647F78E5252409FD12383E906683D9
:100FCE00E0601B123EDBD203E4F50A906578F090E8
:100FDE00668804F0E490667BF0A3F0020A0D90653B
:100FEE007A7404F0906358E0F50A020A0D90668454
:100FFE00E0FF6009F460069080027410F0200E2D60
:10100E00750A02906578E06401FFF090657A7401CC
:10101E00F0EF6005906350800390635463A20190DB
:10102E00668463A2017F04122222020A0D750AC889
:0B103E0090668474FFF0020A0D80FE33
:011049002284
:10002600906379E0B444047F0180027F0090637896
:10003600E0B447047E0180027E00EE5F604A906372
:1000460041E090637AF0906342E090637BF09063C6
:1000560043E090637CF0906344E090637DF09063AE
:1000660045E090637EF0906346E090637FF0906396
:10007600797452F09062B063A2019080A863A201E5
:100086007F06122222020834906334E0C39408509B
:100096000302083D906341E0FF90637AE06F6003DE
:1000A60002083D906342E0FF90637BE06F600302CD
:1000B600083D906343E0FF90637CE06F60030208B5
:1000C6003D906344E0FF90637DE06F600302083D6E
:1000D600906345E0FF90637EE06F600302083D9009
:1000E6006346E0FF90637FE06F600302083D906621
:1000F6008DE060037401F090668E7464F09063790D
:100106007452F0906378E0646D60030202877BFFAF
:100116007A1079741216087BFF7A10798E906341F3
:10012600E0F52EA3E0F52FA3E0F530A3E0F531A32B
:10013600E0F532A3E0F533121608752EFF752F1081
:100146007530EB7531FF7532107533F77BFF7A101A
:1001560079C41216087BFF7A1179001216087BFF04
:100166007A1179651216087BFF7A117991906347A7
:10017600E0F52EA3E0F52FA3E0F530A3E0F531126C
:1001860016087BFF7A1179BB906350E0F52EA3E049
:10019600F52FA3E0F530A3E0F5311216087BFF7AC0
:1001A6001179E9906354E0F52EA3E0F52FA3E0F56D
:1001B60030A3E0F5311216087BFF7A1279179063A7
:1001C6003DE0F52EA3E0F52FA3E0F530A3E0F531F1
:1001D6001216087BFF7A12793A906339E0F52EA35E
:1001E600E0F52FA3E0F530A3E0F5311216087BFF0A
:1001F6007A127957906358E0F52E1216087BFF7A2B
:100206001279881216087BFF7A1279B1A20EE433AE
:10021600F52E1216087BFF7A1279DD906683E0F5DB
:100226002E1216087BFF7A13790A90668DE0F52E5A
:100236001216087BFF7A13793D9062B6E0F52E120E
:1002460016087BFF7A137971A201E433F52E121694
:10025600087BFF7A13799D90667DE0F52EA3E0F585
:100266002FA3E0F530A3E0F531A3E0F532A3E0F5E6
:10027600331216081233617BFF7A1379E8121608D7
:1002860022906378E0644C70527E137FEE122D5AF2
:10029600906380E0F526A3E0F527E4F5287D03AF1B
:1002A60027AE26122E3B7E147F29122D5AAE26AF7C
:1002B60027E4FB7D10122F157E147F2C122D5A7405
:1002C600102527F527E43526F5260528E528C394C5
:1002D6001040CA7E147F2C122D5A22906378E06457
:1002E6006C705CF52A7E147F2E122D5AE4F529AF28
:1002F6002A7E007D03122E3B7E147F29122D5AE49E
:10030600F528A82AE6FF74822528F582E43463F5E9
:1003160083EFF0052A0528E528B410E67E637F8280
:10032600E4FB7D10122F157E147F2C122D5A052901
:10033600E529C3940840B87E147F2C122D5A2290CA
:100346006378E0644B7052F528746A2528F582E4D8
:100356003463F583E06023746A2528F582E4346308
:10036600F583E0FF74802528F582E43463F583E0A5
:10037600B507100528E528B408CF9061047432F05B
:100386000208349063787421F0300A030208347E40
:10039600147F69122D5A020834906378E0B4521A19
:1003A600200A077E147F71122D5A9063787472F0BA
:1003B6007E637F787D081236C022906378E06449B8
:1003C6007045200A077E147F7C122D5A906380E0C8
:1003D600F526A3E0F527E4F528852782852683E020
:1003E600FF74822528F582E43463F583EFF0052750
:1003F600E527700205260528E528B480DC7E637FA4
:10040600787D8A1236C022906378E064437079A3BF
:10041600E064527046200A077E147F84122D5A909B
:100426006380E0F526A3E0F527E4F5288527828595
:100436002683E493FF74822528F582E43463F583EA
:10044600EFF00527E527700205260528E528B48084
:10045600DB7E637F787D8A1236C022906379E06402
:1004660057600302083D906380E0F526A3E0F52778
:1004760074822528F582E43463AD82FC7B80AF2745
:10048600AE26123D05020834906378E064446003AA
:1004960002051F906380E0FF64447003020834EF96
:1004A600B4310CC20A7E147F8D122D5A0208349084
:1004B6006380E0B4300CD20A7E147F99122D5A0262
:1004C6000834906380E0B4320CD20B7E147FA612FF
:1004D6002D5A020834906380E0B4330CC20B7E14AC
:1004E6007FB4122D5A020834906380E0B4340CD2E3
:1004F6000C7E147FC3122D5A020834906380E0B438
:10050600350CC20C7E147FD0122D5A02083490632B
:1005160080E0FF12001E020834906104E070132090
:100526000A077E147FDE122D5A9063787421F0023A
:1005360008349061047432F0906378E0FFB451049B
:10054600C2AF80FEEF64577045200A077E147FEC29
:10055600122D5A906381E0906334F0E4F52890639D
:1005660034E0FFE528C39F4003020834748225283F
:10057600F582E43463F583E0FF906380E025282468
:10058600AFF582E43461F583EFF0052880D09063FF
:1005960078E064536003020642200A077E147FF760
:1005A600122D5A906341E0FF9061B8E06F703C9065
:1005B6006342E0FF9061B9E06F7030906343E0FF03
:1005C6009061BAE0B50724906344E0FF9061BBE018
:1005D600B50718906345E0FF9061BCE0B5070C9045
:1005E6006346E0FF9061BDE06F601690637874210A
:1005F600F0300A030208347E157F06122D5A0208CF
:1006060034E4F528E4F50DAF28FE74AF2528F5820D
:10061600E43461F583E0FD123E770528E528C394AE
:10062600FE40E1C2AFE4907FF0F0A3F0907FFD744E
:10063600AAF0A374FFF0A37455F080FE906378E0EF
:10064600644F704C906380E0F526A3E0F527E5271C
:100656004526700A200A077E157F0F122D5A200A9A
:10066600077E157F16122D5AE4F52874822528F583
:1006760082E43463F583E0852782852683F00527A7
:10068600E527700205260528E528B480DE02083431
:10069600906378E0FFB44521906380E0FDA3E0908D
:1006A6007FF0CDF0A3EDF0C2AF907FFD74AAF0A36A
:1006B60074FFF0A37455F080FEEF646560030208D2
:1006C60034906380E0FFA3E0907FF0CFF0A3EFF0DB
:1006D600E4F526F527D3907FF1E09527907FF0E0AB
:1006E60095264020E4F50D2527FFE5263401FE85F5
:1006F6002782852683E0FD123E770527E5277002CF
:10070600052680D17E157F181235B7EF4E60201270
:100716000003906347EFF0120003906348EFF01276
:100726000003906349EFF012000390634AEFF07EF6
:10073600157F1E1235B7EF4E6020120003906350EE
:10074600EFF0120003906351EFF012000390635232
:10075600EFF0120003906353EFF07E157F241235FD
:10076600B7EF4E6020120003906354EFF0120003BF
:10077600906355EFF0120003906356EFF0120003FA
:10078600906357EFF07E157F2A1235B7EF4E602043
:1007960012000390633DEFF012000390633EEFF00A
:1007A60012000390633FEFF0120003906340EFF0F6
:1007B6007E157F301235B7EF4E602012000390632E
:1007C60039EFF012000390633AEFF01200039063E2
:1007D6003BEFF012000390633CEFF07E157F36127C
:1007E60035B7EF4E6008123BA6906358EFF0E4F57C
:1007F60028E4F50DE5282401FFE433FE74392528A5
:10080600F582E43463F583E0FD123E770528E5289A
:10081600C3944340DCC2AFE4907FF0F0A3F0907F36
:10082600FD74AAF0A374FFF0A37455F080FE7E63F6
:070836007F787D081236C037
:01083D002298
:103CCD00AE07EEC39430400BEED394395005EE247D
:103CDD00D0FF22EEC39461400BEED394665005EEF7
:103CED0024A9FF22EEC39441400BEED39446500518
:083CFD00EE24C9FF22AF0622EC
:103E5D009062AFE004F070069062AEE004F0906204
:0A3E6D00AEE0FEA3E0FF123E41228A
:10000300123E5D123CCDEFC454F0FEC006123E5DBD
:08001300123CCDD0E02FFF22CA
:103BA600123E5D906107EFF0123E5D906108EFF006
:103BB600123E5D906109EFF0123E5D90610AEFF0F2
:103BC600123E5D90610BEFF0123E5D90610CEFF0DE
:103BD600123E5D90610DEFF0123E5D90610EEFF0CA
:103BE600E4A3F0F52EF52FF530F5317B017A6179F6
:053BF600071222F92274
:0435B7008E2B8F2C9C
:1035BB009062AEE4F0A374FFF0123E5DEF606EF428
:1035CB00606B852C82852B83E493B507EC752D01FD
:1035DB00E52C252DF582E4352BF583E493602590BE
:1035EB0062AFE0252DFF9062AEE03400FE123E414B
:1035FB00E52C252DF582E4352BF583E493B50704F3
:10360B00052D80CCE52C252DF582E4352BF583E4B7
:10361B009370A6E52D24FFFFE434FFFE9062AFE02C
:10362B002FF09062AEE03EF07E007F0122E4FEFFC1
:01363B00226C
:102C74007E157F671235B7EF4E70037F01227E15F4
:102C84007F6A1235B7EF4E600C123E5DEF24D024FC
:102C9400FF920E8002D20E7E157F701235B7EF4E72
:102CA400600C123E5DEF24D0906683F08005E490C2
:102CB4006683F07E157F761235B7EF4E600C123EB8
:102CC4005DEF24D090668DF08005E490668DF07EF3
:102CD400157F7C1235B7EF4E600C123E5DEF24D0A9
:102CE4009062B6F08005E49062B6F07E157F8212A1
:102CF40035B7EF4E600C123E5DEF24D024FF9201F5
:102D04008002C20190634163A20190667D63A201C7
:102D14007F0612222230013B7E157F881235B7EFE1
:102D24004E603012000390667DEFF012000390664F
:102D34007EEFF012000390667FEFF01200039066BE
:102D440080EFF0120003906681EFF01200039066AA
:062D540082EFF07F002277
:101D9D00C201E490668DF0D20EC204906683F0907D
:101DAD0062B6F090634163A20190667D63A2017FEC
:101DBD0006122222E4F526E52675F003A4248EF5FD
:101DCD0082E43415F583E493FB740193FA74029362
:101DDD00F91219027003021F8FE4F527F528FD741F
:101DED002F2DF582E43461F583E0FF7003021F8A25
:101DFD00E52675F003A4248EF582E43415F583E40D
:101E0D0093FB740193FA740293F98527827583000D
:101E1D0012191BFEEFB506087528010527021F864E
:101E2D00E5287003021F86EE6003021F81E526245C
:101E3D00FE6028147003021F69147003021F6D14D5
:101E4D007003021F75147003021F792405600302CD
:101E5D001F8A90668D7401F0021F8AD201742F2D96
:101E6D00F582E43461F583E0FF642D7003021F8A6F
:101E7D00123CCDEFC454F0FC74302DF582E4346186
:101E8D00F583E0FF123CCDEF2C90667DF074312D83
:101E9D00F582E43461F583E0FF123CCDEFC454F0DC
:101EAD00FC74322DF582E43461F583E0FF123CCDF4
:101EBD00EF2C90667EF074332DF582E43461F5835A
:101ECD00E0FF123CCDEFC454F0FC74342DF582E4E8
:101EDD003461F583E0FF123CCDEF2C90667FF074FA
:101EED00352DF582E43461F583E0FF123CCDEFC46E
:101EFD0054F0FC74362DF582E43461F583E0FF1265
:101F0D003CCDEF2C906680F074372DF582E4346172
:101F1D00F583E0FF123CCDEFC454F0FC74382DF581
:101F2D0082E43461F583E0FF123CCDEF2C906681A5
:101F3D00F074392DF582E43461F583E0FF123CCD68
:101F4D00EFC454F0FC743A2DF582E43461F583E06E
:101F5D00FF123CCDEF2C906682F08021D204801DC3
:101F6D009066837401F08015C20E80119062B67474
:101F7D0001F08009E4F528F5270D021DEC05260278
:021F8D001DC471
:011F8F00222F
:103C4700906579E0C3947C503D906579E0FE04F07F
:103C570074B72EF582E43462F583EFF0BF0A27903C
:103C67006579E0FF04F074B72FF582E43462F583D9
:103C7700E4F0906579E0FF1237429065797408F0B7
:073C87009062B8E004F02296
:103BFB009080007480F090633963A201F583F582A5
:103C0B0063A2017F0812222290634163A20190807C
:103C1B008863A2017F0A12222290634BE0FF9080FF
:103C2B00B1F09080E1EFF09080957455F0A3F09097
:0C3C3B0080007401F09080097470F02289
:1038B900908009E04410F09080A0E0706C9080A1A5
:1038C9007482F09080A874FFF0A3F0A3F0A3F07FB6
:1038D900039080AEEFF07FCBA3EFF07F039080AC35
:1038E900EFF0A374CBF09080007402F0906AE112BB
:1038F9001A4100000000906AE1E0908040F0906A6F
:10390900E2E0908041F0906AE3E0908042F0906AB2
:10391900E4E0908043F0A3E4F0A3F0A3F0A3F090D7
:093929008018F0A3F0A3F0A3F054
:013932002272
:043AE900AD07AC0673
:103AED00908009E04440F09080D17482F0AF049052
:103AFD0080DEEFF0AF05A3EFF09080027402F0903E
:103B0D006AE5121A4100000000906AE5E0908058C5
:103B1D00F0906AE6E0908059F0906AE7E090805A64
:103B2D00F0906AE8E090805BF0A3E4F0A3F0A3F0DE
:0C3B3D00A3F0908030F0A3F0A3F0A3F000
:013B49002259
:1032BF00908009E04420F09080B8E0600302336012
:1032CF009080B97482F07F039080C6EFF07FCDA31A
:1032DF00EFF07F039080C4EFF0A374CDF03018228D
:1032EF00906350E09080C0F0906351E09080C1F007
:1032FF00906352E09080C2F0906353E09080C3F0EF
:10330F00800C9080C074FFF0A3F0A3F0A3F0908026
:10331F00017402F0906AE9121A4100000000906AED
:10332F00E5E090804CF0906AE6E090804DF0906A76
:10333F00E7E090804EF0906AE8E090804FF0A3E4D1
:10334F00F0A3F0A3F0A3F0908024F0A3F0A3F0A3D8
:01335F00F07D
:01336000224A
:10363C008C268D27A907EAFDE975F018A424ACFFA8
:10364C00E5F034808F82F583EDF0EBFDE975F01831
:10365C00A4FFAEF024ACFBEE34808B82F583A3ED9B
:10366C00F08527828C83E0FDEF24A8FFEE3480FEEA
:10367C008F82F583EDF08527828C83A3E08F828E79
:10368C0083A3F0852782852683A3A3E0FDE975F04B
:10369C0018A424A8FFE5F03480FE8F82F583A3A341
:1036AC00EDF08527828C83A3A3A3E08F828E83A366
:0436BC00A3A3F022B2
:0636C0008D2BAB07AA06EA
:1036C600906AE1E0FCA3E0FDA3E0FEA3E0F52F8E07
:1036D6002E8D2D8C2CAE02AF038E838F8263A201BA
:1036E600E52E540744C0F583852F8263A201AF2BD4
:1036F60012228B908000E020E5F9E4FCFDFEE52F28
:10370600252BF52FEE352EF52EED352DF52DEC3539
:103716002CF52C908040E52CF0A3E52DF0A3E52EAA
:10372600F0A3E52FF09080007420F0AF2FAE2EAD01
:0B3736002DAC2C906AE1121A35AF2B6D
:013741002265
:06383E008D26AB07AA066F
:10384400906AE5E0FCA3E0FDA3E0FEA3E0F52A8E88
:10385400298D288C27AE02AF038E838F8263A20149
:10386400E529540744D0F583852A8263A201AF2653
:1038740012228BE4FCFDFEE52A2526F52AEE3529E5
:10388400F529ED3528F528EC3527F527908058E5FE
:1038940027F0A3E528F0A3E529F0A3E52AF090801A
:1038A400027420F0AF2AAE29AD28AC27906AE51245
:0438B4001A35AF26EC
:0138B80022ED
:023172008F27A5
:10317400908001E030E5037F0022906AE9E0FCA33F
:10318400E0FDA3E0FEA3E0F52B8E2A8D298C289088
:10319400667D63A201E52A540744C8F583852B8222
:1031A40063A2017F061222A1E52B2406F52BE43548
:1031B4002AF52AE43529F529E43528F52890657B94
:1031C40063A201E52A540744C8F583852B8263A2D0
:1031D40001AF271222A1E4FCFDFEE52B2527F52BE8
:1031E400EE352AF52AED3529F529EC3528F5289010
:1031F400804CE528F0A3E529F0A3E52AF0A3E52B0C
:10320400F09080017420F0AF2BAE2AAD29AC289049
:073214006AE9121A35AF2729
:01321B002290
:102B70009081E0E0F5260526052605260526052692
:102B800005260526052605260526908010E0F52950
:102B9000A3E0F52AA3E0F52BA3E0F52C9081E1E07A
:102BA000F5260526052605260526052605260526DD
:102BB000052605260526908014E0F52DA3E0F52EC8
:102BC000A3E0F52FA3E0F530E52FB52B08E530B5F0
:102BD0002C037F0022E4F526E52F540744E0F5831B
:102BE00085308263A20190637863A2017F0812227C
:102BF000B990637A63A2019062B063A2017F06126A
:102C00002222906378E0F527A3E0F528E4F52690EA
:102C10006378E0702AA3E024F8F526E52F540744F2
:102C2000E0F58385308274082582F582E43583F5EA
:102C30008363A20190637863A201AF261222B9AE2A
:102C400027E4FCFDE5302528F530E52F3EF52FED96
:102C5000352EF52EEC352DF52D908014E52DF0A3B5
:102C6000E52EF0A3E52FF0A3E530F090800074404E
:032C7000F0AF269C
:012C7300223E
:102640009081E6E0F52605260526052605260526C1
:1026500005260526052605260526908028E0F5296D
:10266000A3E0F52AA3E0F52BA3E0F52C9081E7E0A9
:10267000F526052605260526052605260526052612
:1026800005260526052690802CE0F52DA3E0F52EE5
:10269000A3E0F52FA3E0F530E4F526E52FB52B0AEE
:1026A000E530B52C05C20802279AE52F540744F0FF
:1026B000F58385308263A20190637863A2017F086D
:1026C0001222B9906378E0F527A3E0F528E52845C4
:1026D0002770099080027410F07F0022906684E0D9
:1026E000FFF4602D90637AE06F7076906685E0FF6E
:1026F00090637BE06F706A906686E0FF90637CE099
:102700006F705E906687E0FF90637DE06F6022806F
:102710005090637AE0906684F090637BE0906685E9
:10272000F090637CE0906686F090637DE090668731
:10273000F0906378E0702AA3E024F8F526E52F54A2
:102740000744F0F58385308274082582F582E435EC
:1027500083F58363A20190637863A201AF261222FE
:10276000B9AE27E4FCFDE5302528F530E52F3EF530
:102770002FED352EF52EEC352DF52DAF2CAE2BADE6
:102780002AAC29AB30AA2FA92EA82DD3121A244087
:10279000099080027410F07F002290802CE52DF0CB
:1027A000A3E52EF0A3E52FF0A3E530F090800274AE
:0427B00040F0AF2620
:0127B4002202
:1027B5009081E3E0F526052605260526052605264E
:1027C5000526052605260526052690801CE0F52903
:1027D500A3E0F52AA3E0F52BA3E0F52C9081E4E036
:1027E500F52605260526052605260526052605269C
:1027F500052605260526908020E0F52DA3E0F52E7B
:10280500A3E0F52FA3E0F530E4F526E52FB52B0A77
:10281500E530B52C05C209022902E52F540744E825
:10282500F58385308263A20190600463A2017F0E67
:102835001222CF906004E0F527A3E0F52890600C04
:10284500E0FFF4604590667DE0FEEF6E7070A3E0FA
:10285500FF90600DE06F706690667FE0FF90600E00
:10286500E06F705A906680E0FF90600FE06F704EE9
:10287500906681E0FF906010E06F7042906682E0A4
:10288500FF906011E06F60068034D291D28D906028
:1028950004E0702AA3E024F2F526E52F540744E866
:1028A500F583853082740E2582F582E43583F583C0
:1028B50063A20190600463A201AF261222CFAE2766
:1028C500E4FCFDE5302528F530E52F3EF52FED3507
:1028D5002EF52EEC352DF52DAF2CAE2BAD2AAC29D2
:1028E500AB30AA2FA92EA82DD3121A245006E528FD
:1028F500452770099080017410F07F002290802098
:10290500E52DF0A3E52EF0A3E52FF0A3E530F0903B
:0729150080017440F0AF26C1
:01291C002298
:042D5A008E2B8F2C01
:102D5E00906AE1E0FCA3E0FDA3E0FEA3E0F5328E75
:102D6E00318D308C2FE532FFE5315407FEE42FF51F
:102D7E002EEE34C0F52D852E82F5837423F0052EAC
:102D8E00E52E7002052D532DC7F582852D83740A0D
:102D9E00F0052EE52E7002052D532DC7906341636D
:102DAE00A201852D83852E8263A2017F0612228BBE
:102DBE007406252EF52EE4352DF52D852B83852CC9
:102DCE008263A201852D83852E8263A20112226F5A
:102DDE00908000E020E5F9E4FCFDFE906AE1E0F869
:102DEE00A3E0F9A3E0FAA3E02FFFEE3AFEED39FDE2
:102DFE00EC38FCEF2408FFE43EFEE43DFDE43CFC31
:102E0E00906AE1121A35906AE1E0908040F0906A83
:102E1E00E2E0908041F0906AE3E0908042F0906AA8
:0C2E2E00E4E0908043F09080007420F0FD
:012E3A002275
:062F15008E2B8F2C8D2D88
:102F1B00906AE1E0FCA3E0FDA3E0FEA3E0F5338EB5
:102F2B00328D318C30E533FFE5325407FEE42FF55B
:102F3B002FEE34C0F52E852F82F5837423F0052FE9
:102F4B00E52F7002052E532EC7F582852E83EBF0ED
:102F5B00052FE52F7002052E532EC790634163A2F8
:102F6B0001852E83852F8263A2017F0612228B742B
:102F7B0006252FF52FE4352EF52E852B83852C82F8
:102F8B0063A201852E83852F8263A201AF2D1222AE
:102F9B008B908000E020E5F97408252DF52DFFE4DA
:102FAB00FCFDFEE5332FF533EE3532F532ED3531E1
:102FBB00F531EC3530F530908040E530F0A3E5315C
:102FCB00F0A3E532F0A3E533F09080007420F0AF6E
:0D2FDB0033AE32AD31AC30906AE1121A35E0
:012FE80022C6
:023742008F3FB7
:10374400906AE1E0FCA3E0FDA3E0FEA3E0F5438E74
:10375400428D418C40E543FFE5425407FEE42FFFD0
:10376400EE34C09062B763A201F5838F8263A20135
:10377400AF3F12228B908000E020E5F9E4FCFDFECF
:10378400E543253FF543EE3542F542ED3541F5413C
:10379400EC3540F540908040E540F0A3E541F0A3CE
:1037A400E542F0A3E543F09080007420F0AF43AE0F
:0B37B40042AD41AC40906AE1121A35B2
:0137BF0022E7
:062E3B008E2B8F2CAB056D
:102E4100906AE1E0FCA3E0FDA3E0FEA3E0F5328E91
:102E5100318D308C2FE532FFE5315407FEE42FF53B
:102E61002EEE34C0F52D852E82F5837423F0052EC8
:102E7100E52E7002052D532DC7F582852D83EBF0CC
:102E8100052EE52E7002052D90634163A201852D6B
:102E910083852E8263A2017F0612228B7406252E62
:102EA100F52EE4352DF52D532DC7E52B852E828585
:102EB1002D83F0052EE52E7002052D532DC7F582C9
:102EC100852D83E52CF0052EE52E7002052D532D61
:102ED100C7908000E020E5F9E532240AF532E435B7
:102EE10031F531E43530F530E4352FF52F90804060
:102EF100E52FF0A3E530F0A3E531F0A3E532F09042
:102F010080007420F0AF32AE31AD30AC2F906AE169
:032F1100121A355C
:012F1400229A
:103E4100E5D220E0FBC2AF438E2075D2028F828E75
:0B3E510083E0FFE4F5D2538EDFD2AF18
:013E5C002243
:103E7700E5D220E0FBC2AF43D2028F828E83EDF002
:093E870075D25063D250D2AF2273
:1037C000E4FDED2401FFE433FE123E4174392DF592
:1037D00082E43463F583EFF00DBD3FE6E4FDED24B4
:1037E0007FFFE433FE123E41742F2DF582E43461F5
:1037F000F583EFF0742F2DF582E43461F583E070EA
:103800001B742F2DF582E43461F5837420F074303D
:103810002DF582E43461F583E4F080040DBD80BEB3
:10382000E49061AEF0FDEDFF7E00123E4174AF2DDD
:0D383000F582E43461F583EFF00DBDFEE993
:01383D002268
:023D05008B2B06
:103D0700A2AF920FC2AF85A22C53A2FE8E838F82E1
:103D170005A28C838D8274091222E7E52B53A2FE3C
:103D270043A2201222E953A2DF852CA2A20F92AF51
:013D3700FF8C
:013D38002268
:103E2400A2AF920FC2AF8C838D82EF1222E743A21E
:0C3E3400201222E953A2DFA20F92AFFF80
:013E4000225F
:023DB8008F2654
:103DBA00A2AF920FC2AFE4F5838D8274061222E796
:103DCA00E52643A2201222E953A2DFA20F92AF7F77
:013DDA0001E7
:013DDB0022C5
:023DDC008F2630
:103DDE00A2AF920FC2AFE4F5838D82740A1222E76E
:103DEE00E52643A2201222E953A2DFA20F92AF7F53
:013DFE0001C3
:013DFF0022A1
:10214700A907E7FFA805EF93C3966008403B74FC17
:102157002FFF80F00F08EF93C3966008402B74FBA6
:102167002FFF80E00F08EF93C3966008401B74FAB7
:102177002FFF80D00F08EF93D3966008400B74F9B8
:102187002FFF80C01F1F1F1F1FEF54FEF80303F709
:10219700E893FC08E893FD08E893FE08E893FF221C
:1021A70009E993C39D6008402974FB29F980F10967
:1021B700E993C39E6008401A74FA29F980E209E995
:1021C70093D39F6008400B74F929F980D319191923
:1021D7001919E9C313C313FF22740093F8ECC398CA
:1021E7004024701F740193F8EDC39840197014745C
:0E21F7000293F8EEC398400E7009740393F83B
:10220500EFC39840037F00227F0122EDF8E6F00836
:10221500A3DFFA22EDF8E0F608A3DFFA22E0A363D4
:10222500A201F0A363A201DFF475A20022E0A3637B
:10223500A201F0A363A201E0A363A201F0A363A23C
:1022450001E463A201F0A363A201DFE175A200220C
:10225500E0A363A2016DFE936CFDEE058393FC156F
:102265008363A201DFEA75A200227F00E493A363E2
:10227500A201F00F600CA3E583C2E3F58363A2011D
:1022850080EA75A20022E0A363A201F0A3E583C260
:10229500E3F58363A201DFEE75A20022E0A363A24A
:1022A50001F0A3E583C2E4D2E3F58363A201DFEC89
:1022B50075A20022E583C2E3F583E0A363A201F0E2
:1022C500A363A201DFEE75A20022E583C2E4D2E397
:1022D500F583E0A363A201F0A363A201DFEC75A27D
:1022E5000022F922C002C004C00612FFF0D006D0B9
:0422F50004D00222ED
:103C8E000A536572763A00200A4441544147524124
:103C9E004D3A200020547261737353656E64455221
:103CAE00520A00205265496E69742043414E0A0043
:0F3CBE002043414E283029203E20544F210A0038
:03001E00E4FF22DA
:103D6C00C28DC2AF438901C28C9069D7E0FF700746
:103D7C00F58A758CEE800AEFB40A06E4F58A758C28
:063D8C0070D28CD2AF22C0
:103D3900C28DC2AF438901C28C9069D7E0FF70146C
:103D4900302309F58A758CDCC2238012758A667561
:103D59008CFC800AEFB40A06E4F58A758CDCD28CF7
:033D6900D2AF22B4
:103D9200C2249069D7E0C394645006123A21123DBE
:103DA2006C120022D222E4F558906ADFF0F544F555
:063DB2005DC223F55B2257
:102A4F00EF24FCF526200A127E3C7F8E122D5A7E33
:102A5F00637F7CE4FBAD26122F1590637BE0641F30
:102A6F006003022B56D224906378E0B40108C22091
:102A7F00AF261239332290637EE064087037906A74
:102A8F005F7442F0A37418F090637CE0906A61F079
:102A9F0090637DE0906A62F0A37408F090637F63A7
:102AAF00A201906A6463A201FF12222275440DE411
:102ABF00F555C2202290637EE0FFB40A1D906A5F35
:102ACF007401F0A37418F0A37480F0A3740AF0E4F7
:102ADF00A3F0754405F555C22022EFB40B1D906A83
:102AEF005F7401F0A37418F0A37480F0A37409F05D
:102AFF00E4A3F0754405F555C22022EFB40D1D90E7
:102B0F006A5F7401F0A37418F0A37480F0A3740BC0
:102B1F00F0E4A3F0754405F555C22022EF64077069
:102B2F003F906A5F04F0A37418F0A37480F0A3744D
:102B3F000CF0A37401F090637FE0906A64F0754429
:102B4F0006E4F555C2202290637C63A201906A5F70
:102B5F0063A201AF26122222852644E4F555C22036
:012B6F002243
:0F3EA700D3EF6480948E5006E55D70028F5D222C
:101B7300208D03021C2BC28C202203021D00E55D75
:101B8300602F9060047D46FF122219123D6C123BB8
:101B93004AC291200A077E3C7F95122D5A200A0BD8
:101BA3007E607F04E4FBAD5D122F15E4F55D021D3D
:101BB30000E544605474632555F582E4346AF58383
:101BC300E02405F526D3940E4008E4F544D2200220
:101BD3001D00745F2555F582E4346AF5837D46AFB5
:101BE30026122219E5262555F555E54630E702D29A
:101BF30023123D6C123B4AE555C395445003021D25
:101C030000E4F544D220021D00E55A60159069C333
:101C13007D46FF122219123D6C123B4AE4F55A022B
:101C23001D00123A86123D6C12291D8F26EF700398
:101C3300021D00123D39E4F55BE55CC3946E40037D
:101C4300021CD9302466E54664427060E54A70237D
:101C530085484685494775480874D8255CF582E46C
:101C63003469F5837403255CF55C7D467F0312229A
:101C730010806374D8255CF582E43469F583E52626
:101C8300255CF55C7D46AF26122210300C48C3E577
:101C93005C9526FFE49400FE74D82FF58274693EA8
:101CA300AF82FEE4FBAD26122F15802AE546B4422F
:101CB3000DE549B402089062B6E06401601874D877
:101CC300255CF582E43469F583E526255CF55C7DC6
:101CD30046AF26122210300124E54630E7033018C0
:101CE3001C90657B7D46AF26122210AF26123172FF
:101CF300EF700A200A077E3C7FA2122D5A300D1A7C
:101D03003000159069D7E0C39464500C055BE55B24
:101D130094F04004C2AF80FEC20D300279E55860F2
:101D230031D39401400415588028906ADFE004F011
:101D3300E0D39403400D200A077E3C7FB1122D5A55
:101D4300123D92200A077E3C7FBE122D5AE4F558BD
:101D5300D222E55A703E0557E557B556189069C328
:101D63007401F0A37408F0A37480F0A37408F0E482
:101D7300A3F0755A05E557B5591AE4F5579069C3A9
:101D830004F0A37408F0A37480F0A37407F0E4A331
:091D9300F0755A05C20212321C5F
:011D9C002224
:1039AC00E5146033E4F51490647804F0A37403F028
:1039BC0090667CE090647AF0A3741FF09067C1E08D
:1039CC0090647CF09067C2E090647DF09067C3E0F7
:1039DC0090647EF07F0122E55C6037E4906478F0BF
:1039EC00A3E55CF090667CE090647AF0302406A34A
:1039FC00741FF0800690647B7419F09069D863A2F0
:103A0C000190647C63A201AF5C122222E4F55C7F1E
:053A1C0001227F0022E1
:0B3EB600302005C2207F01227F002287
:0100210022BC
:063EDB00E4F55CF5442251
:0A3EC100E4906107F0A3F0A3F022E3
:103E00002043616E457247495400200A00204361F7
:103E10006E457272434821000A000A2052657145BE
:043E20007272210099
:10291D00E59B541F6020200A1A7E3E7F00122D5A1F
:10292D00E59B541FFF7E007D03122E3B7E3E7F0AEA
:10293D00122D5AE4F59BE5BA30E010E4F5B375B10C
:10294D0080F5B2D222F558906ADFF0E5CFF470032E
:10295D00022A4C752801E4F527E5CFF455287003BC
:10296D00022A3AE527C454F0F5B1E5B2547F64204C
:10297D006003022A0BE5B3540FF54A85BC462018B7
:10298D0016E5BD541FFF131313541FFFE5BD54E08F
:10299D0044184FF5478006E5BD54E0F547E5BDC445
:1029AD003354E0FFE5BE131313541F4FF548E5BE36
:1029BD00C43354E0FFE5BF131313541F4FF549857E
:1029CD00A34B85A34C85A34D85A34E85A34F85A30E
:1029DD005085A35185A352E4F5B230180C85AE5342
:1029ED0085AF5475B3D07F0F22E546547EB54605AD
:1029FD0075B350800375B3D0E54A2405FF22E5B2C7
:102A0D00549F6023200A207E3E7F0D122D5AAFB2B7
:102A1D007E007D03122E3BAFB37E007D03122E3B55
:102A2D007E3E7F18122D5AE4F5B275B3D0E52825F8
:102A3D00E0F5280527E527C3940850030229667F92
:012A4D000088
:012A4E002265
:103B4A0020185875B180E4F5B3F5B28546BCE5484E
:103B5A00C4135407FFE54754E04FF5BDE548333336
:103B6A003354F8FFE549C41354074FF5BEE549330A
:103B7A00333354F8F5BF854BA3854CA3854DA385F4
:103B8A004EA3854FA38550A38551A38552A3E54A29
:0C3B9A00540F2450F5B375580AC22222C3
:103A860020185F75B190E5B220E613200A107E3E3D
:103A96007F1A122D5AAFB27E007D03122E3BE4F53B
:103AA600B3F5B274912516F582E43467F583E0F533
:103AB600BCE4F5BD74922516F582E43467F583E01F
:103AC600FF33333354F8F5BE75BF78051605167403
:103AD600912516F582E43467F583E07002F51675D4
:033AE600B35022B8
:093ECB00EF6003C29622D2962298
:103A210043AB01C2E8C2EAE4FFEFC454F0F5B1C30D
:103A3100EF64809488500575B3D08003E4F5B3E456
:103A4100F5B2F5BCF5BDF5BEF5BFF5C4F5C5F5C6D6
:103A5100F5C7F5A3F5A3F5A3F5A3F5A3F5A3F5A381
:103A6100F5A30FBF0EC39069D7E0FF25E0F5B4754C
:103A7100B50C75B66C75A11275AB0275C13E75C3F7
:043A8100FF75C20308
:013A8500221E
:101F90003E2A2C312CCFE0F0E0ECE5F2F0FB20E41F
:101FA000E8F1EFE5F2F7E5F0F1EAE8E3EE20F9E831
:101FB000F2E00A003E4C2C4930312C256C752CD1B6
:101FC000EAEEF0EEF1F2FC20EEE1ECE5EDE020EDE2
:101FD000E020F8E8EDE52052533438352C3132302A
:101FE000302C323430302C343830302C39363030DC
:101FF0002C31393230302C33383430302C353736C0
:1020000030302C3131353230300A003E4C2C4930E2
:10201000322C25732C43EAEEF0EEF1F2FC20EDE0D9
:1020200020F8E8EDE52043414E2C30202D203530BE
:1020300030EAE1283530EC292C31202D203530EAEA
:10204000E128353030EC292C32202D20D8E8EDE085
:1020500020EEF2EBFEF7E5EDE00A0030202D203512
:102060003030EAE1283530EC290031202D203530A0
:10207000EAE128353030EC290032202D20D8E8ED77
:10208000E020EEF2EBFEF7E5EDE0003E532C4930A8
:10209000332C2562752CCFE5F0E8EEE420E8EDE482
:1020A000E8EAE0F6E8E820282A3130ECF129283C7B
:1020B000323530290A003E532C4930342C256275C4
:1020C0002CCFE5F0E8EEE420ECEEF0E3E0EDE8FF05
:1020D00020282A3130ECF129283C323530290A00F9
:1020E0003C21003C4930313D003C4930323D003C10
:1020F0004930333D003C4930343D005452414E5A42
:10210000004359434C4500424C494E4B0044454C1A
:102110004159004E4F4B5654004B5000424F4F54C4
:102120000043414E00000A4F55543A00FF20FBFF88
:102130002101FF2107FF210DFF2113FF2119FF219D
:072140001CFF2121FF2125F6
:103361007BFF7A1F79901216089069C1E0FEA3E0F5
:10337100FFC3E49FFFE49EFEAB07FA3395E0F9F843
:103381007F007E8C7D0A7C001219848F318E308DF6
:103391002F8C2E7BFF7A1F79B41216089069D7E023
:1033A1007012752EFF752F2075305B7BFF7A2079A7
:1033B1000B1216089069D7E0B40A12752EFF752F0B
:1033C1002075306A7BFF7A20790B1216089069D735
:1033D100E0B46412752EFF752F207530797BFF7A6A
:1033E10020790B1216087BFF7A20798B85592E12D2
:0F33F10016087BFF7A2079B685562E1216082211
:103496007E207FE01235B7EF4E70037F01227E203B
:1034A6007FE31235B7EF4E6023123BA6A804A905A9
:1034B600AA06AB077F007E8C7D0A7C001219841257
:1034C6001A169069C1EEF0A3EFF0800A9069C174F4
:1034D600FFF0A374B8F0E49069D7F07E207FE9127C
:1034E60035B7EF4E6015123E5DBF31069069D77451
:1034F6000AF0BF32069069D77464F07E207FEF121F
:1035060035B7EF4E6007123BA68F59800375596495
:103516007E207FF51235B7EF4E6006123BA68F561A
:043526002275565A5A
:01352A00227E
:03002300022FE9C0
:0D2FE900C0E0C0F0C083C082C0D075D01819
:102FF600309844C298750B01AF9920190BEF640203
:103006007035D219D291802F301C07C21C531F0F66
:103016008016BF0904D21C801EBF030C85101475D0
:103026001000C219C291800F74C12510F582E434D4
:1030360067F583EFF0051030996F301A6AE512B420
:10304600FF0C7599020512751500D2908059E5128C
:10305600B50F077599030512804DE512D3950F40FC
:103066000FC21AD21EE4FF123ECBD220C290803786
:10307600E5156009F5990512751500802A74C125B4
:1030860012F582E43468F583E0F5156402600BE519
:103096001564036005E515B4090575990980088569
:0930A60015990512751500C29977
:0B30AF00D0D0D082D083D0F0D0E0322F
:10249D00E4906AEDF0906AEDE075F003A4242CF55C
:1024AD0082E43421F583E493FB740193FA7402936F
:1024BD00F9121902700302263FE4906AEFF0A3F0BF
:1024CD00906AEEF0906AEEE0242FF582E43461F527
:1024DD0083E0FF7003022636906AEDE075F003A4E9
:1024ED00242CF582E43421F583E493FB740193FAF3
:1024FD00740293F9906AEFE0F58275830012191B4F
:10250D00FEEFB5060F906AF07401F0906AEFE004EB
:10251D00F002262D906AF0E0700302262DEE600386
:10252D00022624906AEDE01460611470030225C642
:10253D0024FB70030225F424076003022636906AFB
:10254D00EEE0242FF9E43461FA7B01C0031B8B2EDE
:10255D00752F00753000E4F531D0031222F9906A21
:10256D00F1121A35906AF1E0F8A3E0F9A3E0FAA3AD
:10257D00E0FB7F007E8C7D0A7C00121984121A16F6
:10258D009069C1EEF0A3EFF0022636906AEEE024DA
:10259D002FF9E43461FA7B01C0031B8B2E752F00DC
:1025AD00753000E4F531D0031222F9906AF1121A58
:1025BD0035906AF4E0F5598070906AEEE0242FF9B9
:1025CD00E43461FA7B01C0031B8B2E752F0075302F
:1025DD0000E4F531D0031222F9906AF1121A359008
:1025ED006AF4E0F5568042906AEEE0242FF9E43467
:1025FD0061FA7B01C0031B8B2E752F00753000E433
:10260D00F531D0031222F9906AF1121A35906AF45D
:10261D00E09069D7F08012E4906AF0F0906AEFF0E4
:10262D00906AEEE004F00224D1906AEDE004F0022D
:02263D0024A2D5
:01263F002278
:1030BA00E4FF123ECBC21AC21EC219C21CE4F512A8
:1030CA00F50FF510F50B9069C174FFF0A374F4F0D5
:1030DA00E4906790F0A374C2F0E4A3F0A374C2F082
:1030EA00A37401F0A374C2F0A37402F0A374C2F033
:1030FA00A37403F0A374C2F0A37404F0A374C2F01F
:10310A00A37405F0A374C2F0A37406F0A374C2F00A
:10311A00A37407F0E4A3F0A3F0C218F5169069D7D8
:10312A00F075596475565A123496EF600312249D4D
:10313A00E4F511C2ADF5C9D2CDD2CCC2C9C2CAF525
:10314A00CDF5CC9069C1E0F5CBA3E0F5CA85CBCD2E
:10315A0085CACCD29ED29CD2CAC2ACC298C2997538
:08316A00B81075B710D2AC22B9
:0100220022BB
:023933008F27DC
:10393500301A03C22022E4FFFEEEC39527502874F7
:103945007C2EF582E43463F583E0FD74C12EF582A7
:10395500E43468F583EDF074C12EF582E43468F53E
:1039650083E02FFF0E80D2EFF4FF74C12527F58287
:10397500E43468F583EFF07F01123ECBE52704F5CB
:103985000FD21B200A127E217F26122D5A7E687FB8
:10399500C1E4FBAD0F122F157512FFD21AC2992083
:0639A50099FDD299C21E3B
:0139AB0022F9
:10321C002000030232A8C200906790E004F0E0B4F2
:10322C00051DE490637CF0A3F0A3742EF0A374341A
:10323C00F0A304F0A304F0A304F07F071239339039
:10324C006790E0B40A23E490637CF0A3F0A3742E9F
:10325C00F0A314F0A37438F0A3742EF0A37439F017
:10326C00A37433F07F08123933906790E0D3940F36
:10327C004024E4F090637CF0A3F0A3742EF0A374CC
:10328C0020F0A37431F0A304F0A3742EF0A37433D4
:10329C00F07F0812393390678FE004F0301A0E90EB
:1032AC00678FE0D39414400AC21AD21E22E49067AE
:0332BC008FF0226E
:1035370002083EE493A3F8E493A34003F68001F264
:1035470008DFF48029E493A3F85407240CC8C33395
:10355700C4540F4420C8834004F456800146F6DF64
:10356700E4800B0102040810204080903ED4E47EE2
:10357700019360BCA3FF543F30E509541FFEE49359
:10358700A360010ECF54C025E060A840B8E493A320
:10359700FAE493A3F8E493A3C8C582C8CAC583CA4B
:1035A700F0A3C8C582C8CAC583CADFE9DEE780BE03
:013EDA0000E7
:10190200BB010689828A83E0225002E722BBFE02E3
:09191200E32289828A83E4932216
:10191B00BB010CE58229F582E5833AF583E0225081
:10192B0006E92582F8E622BBFE06E92582F8E222CB
:0D193B00E58229F582E5833AF583E49322E5
:1019480075F008758200EF2FFFEE33FECD33CDCC56
:1019580033CCC58233C5829BED9AEC99E5829840D9
:101968000CF582EE9BFEED9AFDEC99FC0FD5F0D6B6
:10197800E4CEFBE4CDFAE4CCF9A88222B800C1B9E0
:101988000059BA002DEC8BF084CFCECDFCE5F0CB1E
:10199800F97818EF2FFFEE33FEED33FDEC33FCEB57
:1019A80033FB10D703994004EB99FB0FD8E5E4F912
:1019B800FA227818EF2FFFEE33FEED33FDEC33FCFF
:1019C800C933C910D7059BE99A4007EC9BFCE99AF3
:1019D800F90FD8E0E4C9FAE4CCFB2275F010EF2F38
:1019E800FFEE33FEED33FDCC33CCC833C810D70738
:1019F8009BEC9AE899400AED9BFDEC9AFCE899F873
:0E1A08000FD5F0DAE4CDFBE4CCFAE4C8F92205
:0E1A1600C3E49FFFE49EFEE49DFDE49CFC22E1
:101A2400EB9FF5F0EA9E42F0E99D42F0E89C45F018
:011A3400228F
:0C1A3500ECF0A3EDF0A3EEF0A3EFF02224
:101A4100A8828583F0D083D082121A58121A5812B4
:101A51001A58121A58E473E493A3C583C5F0C583D9
:101A6100C8C582C8F0A3C583C5F0C583C8C582C8EF
:011A71002252
:1015A600E53A242EF8E6053A22782B301602782EF4
:1015B600E475F001121AD3021902200FEB7F2ED226
:1015C6000F8018EF540F2490D43440D4FF30130BFF
:1015D600EF24BFB41A0050032461FFE53B600215F7
:1015E6003B053EE53E7002053D30160D782BE47551
:1015F600F001121AD3EF021A72023C477403D21694
:101606008003E4C216F53A8B2B8A2C892DE4F53B30
:10161600F53DF53EE53B60077F201215E180F57547
:101626003CFFC210C20FC211C212C214C215C217A9
:101636001215AFFF700D3016057F001215F2AF3E82
:10164600AE3D22B4255FC2D5C2131215AFFF24D01A
:10165600B40A00501A75F00A783B30D50508B6FF73
:101666000106C6A426F620D5047002D21280D9241B
:10167600CFB41A00EF5004C2E5D2130217F2D2100B
:1016860080C6D20F80C0D21180BCD2D580BAD21407
:1016960080B47F201215E12011077401B53B00408C
:1016A600F11215A6FF1215E102161AD217D21580ED
:1016B600951215A6FB1215A6FA1215A6F94A4B7035
:1016C6000679C37A187BFF20112EE53B602A7E003F
:1016D6008E8275830012191B60060EEE653C70F053
:1016E600C2D5EBC0E0EAC0E0E9C0E0EE121839D09E
:1016F600E0F9D0E0FAD0E0FB121902FF60AAEBC0D5
:10170600E0EAC0E0E9C0E01215E1D0E02401F9D03A
:10171600E03400FAD0E0FBE53C0460DCD53CD9803F
:10172600877BFF7A187935D211809C7910800279EF
:1017360008C215C2178008D2D5790A8004790AC270
:10174600D5E53C047002F53CE4FAFDFEFF1215A651
:10175600FC7B082010131215A6FD7B10300F0A1211
:1017660015A6FE1215A6FF7B20EC3382D592D55026
:1017760013C3E4300F069FFFE49EFEE42010039D92
:10178600FDE49CFCE4CBF8C210EC700CCFCECDCCC3
:10179600E824F8F870F38017C3EF33FFEE33FEED5D
:1017A60033FDEC33FCEB33FB994002FB0FD8E9EB3E
:1017B600301005F8D0E0C448B210C0E00AEC4D4E37
:1017C6004F78207B0070C2EAB53C0040BCC0E012F6
:1017D600183BD0F0D0E0201004C4C0E0C4B210C062
:1017E600F01215CAD0F0D5F0EB02161A121B3216FB
:1017F600B75317315816884C16844217354F173D84
:0F18060044173D49169D4317435517274617278B
:101815004517274718E350168C2D16902E16B32B17
:1018250016942316B12018CC2A164C48000016AB86
:101835003F3F3F00790AA2D5201214301409B91090
:10184500020404B9080104A2D520150250010420A0
:1018550011689211B53B005034C0E07F2030121959
:101865007F30A21172157214500F121892C211C254
:1018750015C214C2177F30800F301403E9C0E0127F
:1018850015E1301403D0E0F9D0E0B53BCC301417A6
:101895007F30B9100C1215E17F583013077F78801F
:1018A50003B908031215E13011057F2D0215E17FFB
:1018B500202017F87F2B2015F322921180CF286E58
:1018C500756C6C2900D2101215A63010F8C210786C
:1018D5003B30D50108F602164C2D504349581215D8
:1018E500A62403B405004001E49018DE931215D236
:0D18F500743A1215D2D212753B040217315D
:1022F9008B2B8A2C892DE4F537F536F535F534F530
:1023090032F533E52F4530452E6012EBC0E0EAC0C7
:10231900E0E9C0E0AB2EAA2FA930121AE3AB2B05D6
:102329002DE52DAA2C7002052C14F9121902F53885
:10233900C394094007E538D3940D40E1E53864209A
:1023490060DBE538B42D054333038016E538B42B3B
:1023590005433301800C74FF252DF52D74FF352CB1
:10236900F52CE53160046410703FAB2BAA2CA92D24
:1023790012190264306009E531702E75310A80291D
:1023890090000112191BFF64786004EFB4581343DD
:1023990033017531107402252DF52DE4352CF52CFA
:1023A9008007E5317003753108AB2B052DE52DAAA2
:1023B9002C7002052C14F9121902F538C3946140E6
:1023C9000AE538D3947A50035338DF74D02538F5A9
:1023D90038C3940A400CE5389411406D74F92538D6
:1023E900F538E538D39531506043330185373C855D
:1023F900363B85353A853439AF317E00E4FCFDAB97
:1024090037AA36A935A834121A84C8ECC8C9EDC947
:10241900CAEECACBEFCBE4FCFDFEEB2538F537EE6F
:102429003AF536ED39F535EC38F534AF37AE36AD2A
:1024390035FCAB3CAA3BA93AA839D3121A2450035C
:102449000223B24333040223B2E53320E003E480DC
:102459002DE52F4530452E601EAB2BE52D24FFF9C8
:10246900E52C34FFFAEBC0E0EAC0E0E9C0E0AB2EAE
:10247900AA2FA930121AE3E53330E20774FFFFFEF1
:10248900FDFC22E533AF37AE36AD35AC3430E10370
:04249900021A1622EB
:101A7200BB010689828A83F0225002F722BBFE0153
:021A8200F3224D
:101A8400E88FF0A4CC8BF0A42CFCE98EF0A42CFC01
:101A94008AF0EDA42CFCEA8EF0A4CDA8F08BF0A47F
:101AA4002DCC3825F0FDE98FF0A42CCD35F0FCEBDE
:101AB4008EF0A4FEA9F0EB8FF0A4CFC5F02ECD39A3
:0F1AC400FEE43CFCEAA42DCE35F0FDE43CFC2210
:101AD300FAE6FB0808E6F925F0F618E6CA3AF62214
:101AE300BB011A89828A83D0F0D0E0F8D0E0F9D024
:101AF300E0FAD0E0FBE8C0E0C0F0021B615016E959
:101B0300F8D083D082D0E0F9D0E0FAD0E0FBC082F5
:101B1300C083021B58BBFE16E9F8D083D082D0E005
:0F1B2300F9D0E0FAD0E0FBC082C083021B6A2237
:101B3200D083D082F8E4937012740193700DA3A342
:101B420093F8740193F5828883E473740293686056
:061B5200EFA3A3A380DF56
:091B5800EBF608EAF608E9F622B2
:091B6100EBF0A3EAF0A3E9F02285
:091B6A00EBF208EAF208E9F222AC
:00000001FF
